:020000040000FA
:0A0000000000000025EF00F033D0EF
:0800180080D0096A086EFF0E9A
:100020000826092200D0D8A01200030E076EE60EA3
:1000300002D8F5D7076AFE0F066EE86A075AD8A0FD
:1000400012000000060600D0F8D74F0EAF6E240E47
:10005000AC6E900EAB6E00010F0EC16E070EB46E4B
:10006000C69A400E926EE00E936EC00E946E6CD0E7
:10007000F2A403D0F294817A11009EAA19D0060E40
:10008000AB1412E1E2CF6EF0E1CF6DF06F2A11EE0A
:1000900000F06F50E126000EE222AECFE7FF6EC007
:1000A000E2FF6DC0E1FF1100AE50AE50AB98AB88DF
:1000B00011006F50705C14E0702AEACF07F0E9CFAE
:1000C00006F001EE00F07050E926000EEA22EF5033
:1000D000066E07C0EAFF06C0E9FFD880120004D010
:1000E000E868066ED8A0120012006F6A706A9D8AD6
:1000F0009F8AF28EF28C12009D9A01EE00F0010EA2
:10010000F46EF36AF306000EF45AEE6AF450F3103C
:10011000F9E16F6A706A9D8A1200F29EE0CF92F454
:10012000D8CF93F4E8CF94F4F28E0001A192F29E1E
:1001300092C4E0FF93C4D8FF94C4E8FFF28E10008D
:100140009EA8FED7AD6E1200939A8A8A0A0E65DFCA
:10015000939A8A9A929489949296899694908B9085
:1001600094928B9294988B98949A8B9A93948A9465
:1001700093968A9692908990929289929298899871
:10018000929A899A94948B9494968B9693908A9051
:1001900093928A9293988A98716A396A376A00EEC4
:1001A00072F0200EEE68E82EFDD7386A5A6A5B6A54
:1001B0005C6A5D6A5E6A5F6A606A616A3B6A3A6A43
:1001C0003D6A3C6A3F6A3E6A416A406A436A426AE3
:1001D000456A446A476A466A496A486A4B6A4A6A93
:1001E0004D6A4C6A4F6A4E6A516A506A536A526A43
:1001F000556A546A576A566A596A586A05EC08F093
:1002000074DF7ADFCD6AF294F28A870ED56EB16A16
:10021000A192A082D08EA292B10EB16E86EC08F0AF
:1002200086EC0AF0662AE86A66B2010F67B0010838
:1002300006E16770622A000E63226422652239DFBC
:100240000A6EB50E0A5C06E3FE0E0A5C01E20C6A59
:100250001DEF04F00AAE22D00C6A840E0A5C05E1A0
:100260000AC00CF00D680E6817D0940E0A5C05E108
:100270000AC00CF00F6810680FD0A40E0A5C05E1EC
:100280000AC00CF01168126807D0B40E0A5C04E1D1
:100290000AC00CF0136814681BEF04F00C5204E160
:1002A0001DEF04F01BEF04F0840E0C5CD8A445D0C5
:1002B0000D2803E10AC00DF03CD00AC00EF03A0E42
:1002C0000D5C04E137903990899430D03B0E0D5C81
:1002D00004E137923992899629D03C0E0D5C04E1F5
:1002E000379439948B9022D03D0E0D5C04E1379603
:1002F00039968B921BD03E0E0D5C04E137983998ED
:100300008B9814D03F0E0D5C04E1379A399A8B9A82
:100310000DD0400E0D5C04E1379C399C8A9406D0C8
:10032000410E0D5C03E1379E399E8A960D681BEFE6
:1003300004F01DEF04F01BEF04F0940E0C5CD8A445
:1003400000EF04F00F2804E10AC00FF0FEEF03F005
:100350000AC010F010523EE13A0E0F5C04E13790F3
:100360003990899433D03B0E0F5C04E13792399277
:1003700089962CD03C0E0F5C04E1379439948B9015
:1003800025D03D0E0F5C04E1379639968B921ED036
:100390003E0E0F5C04E1379839988B9817D03F0ECA
:1003A0000F5C04E1379A399A8B9A10D0400E0F5C9B
:1003B00004E1379C399C8A9409D0410E0F5C04E11A
:1003C000379E399E8A9602D01DEF04F01BEF04F091
:1003D000FEEF03F03A0E0F5CD8A43ED071B002D00D
:1003E000898001D0899071708984378002EE92F003
:1003F000D8901034E926000EEA22EECF4AF0EFCF73
:100400004BF04A506224006E4B506320016E000E88
:100410006420026E000E6520036E03C075F002C0FA
:1004200074F001C073F000C072F05A5213E03980CA
:1004300003EE92F0D8905A34E926000EEA22EECF6D
:1004400000F0EFCF01F04A50005C3A6E4B5001587B
:100450003B6E01D03990D0D13B0E0F5CD8A43ED07A
:1004600071B202D0898201D08992717289863782F5
:1004700002EE92F0D8901034E926000EEA22EECF78
:100480004CF0EFCF4DF04C506224006E4D50632085
:10049000016E000E6420026E000E6520036E03C024
:1004A00079F002C078F001C077F000C076F05B52BE
:1004B00013E0398203EE92F0D8905B34E926000E07
:1004C000EA22EECF00F0EFCF01F04C50005C3C6E22
:1004D0004D5001583D6E01D039928ED13C0E0F5CCB
:1004E000D8A43ED071B402D0898801D089987174A3
:1004F0008B80378402EE92F0D8901034E926000EFB
:10050000EA22EECF4EF0EFCF4FF04E506224006E55
:100510004F506320016E000E6420026E000E6520B5
:10052000036E03C07DF002C07CF001C07BF000C010
:100530007AF05C5213E0398403EE92F0D8905C3488
:10054000E926000EEA22EECF00F0EFCF01F04E5088
:10055000005C3E6E4F5001583F6E01D039944CD133
:100560003D0E0F5CD8A43ED071B602D0898A01D06E
:10057000899A71768B82378602EE92F0D890103489
:10058000E926000EEA22EECF50F0EFCF51F05050A6
:100590006224006E51506320016E000E6420026ED2
:1005A000000E6520036E03C081F002C080F001C020
:1005B0007FF000C07EF05D5213E0398603EE92F0CA
:1005C000D8905D34E926000EEA22EECF00F0EFCF9E
:1005D00001F05050005C406E51500158416E01D006
:1005E00039960AD13E0E0F5CD8A43ED071B802D025
:1005F0008B8401D08B9471788B88378802EE92F0CF
:10060000D8901034E926000EEA22EECF52F0EFCF58
:1006100053F052506224006E53506320016E000E5E
:100620006420026E000E6520036E03C085F002C0D8
:1006300084F001C083F000C082F05E5213E039887C
:1006400003EE92F0D8905E34E926000EEA22EECF57
:1006500000F0EFCF01F05250005C426E5350015851
:10066000436E01D03998C8D03F0E0F5CD8A43ED05D
:1006700071BA02D08B8601D08B96717A8B8A378AB9
:1006800002EE92F0D8901034E926000EEA22EECF66
:1006900054F0EFCF55F054506224006E5550632053
:1006A000016E000E6420026E000E6520036E03C012
:1006B00089F002C088F001C087F000C086F05F5268
:1006C00013E0398A03EE92F0D8905F34E926000EE9
:1006D000EA22EECF00F0EFCF01F05450005C446E00
:1006E00055500158456E01D0399A86D0400E0F5CA6
:1006F000D8A43ED071BC02D08A8001D08A90717C8F
:100700008A84378C02EE92F0D8901034E926000EDD
:10071000EA22EECF56F0EFCF57F056506224006E2B
:1007200057506320016E000E6420026E000E65209B
:10073000036E03C08DF002C08CF001C08BF000C0CE
:100740008AF0605213E0398C03EE92F0D890603456
:10075000E926000EEA22EECF00F0EFCF01F056506E
:10076000005C466E57500158476E01D0399C44D00A
:10077000410E0F5CD8A43ED071BE02D08A8201D057
:100780008A92717E8A86378E02EE92F0D89010346B
:10079000E926000EEA22EECF58F0EFCF59F058507C
:1007A0006224006E59506320016E000E6420026EB8
:1007B000000E6520036E03C091F002C090F001C0EE
:1007C0008FF000C08EF0615213E0398E03EE92F08C
:1007D000D8906134E926000EEA22EECF00F0EFCF88
:1007E00001F05850005C486E59500158496E01D0D4
:1007F000399E02D00F6821D00F681DD01ED01BD0AB
:10080000A40E0C5C0BE1112803E10AC011F004D026
:100810000AC012F07DEC06F010D00DD0B40E0C5CC6
:100820000AE1132803E10AC013F004D00AC014F04F
:1008300038EC07F002D043EC06F0080E6C5CD8B040
:100840003BEF06F06850625C695063586A50645828
:100850006B506558D8A000D26B8E6C523DE18994E4
:1008600039B005D0756874687368726834D037A081
:1008700016D03A506224006E3B506320016E000E89
:100880006420026E000E6520036E03C075F002C086
:1008900074F001C073F000C072F037901CD071B0DA
:1008A00002D0898001D08990898471704A50622475
:1008B000006E4B506320016E000E6420026E000E2D
:1008C0006520036E03C075F002C074F001C073F0C0
:1008D00000C072F03780BFD1010E6C5C3DE189969B
:1008E00039B205D0796878687768766834D037A2ED
:1008F00016D03C506224006E3D506320016E000E05
:100900006420026E000E6520036E03C079F002C001
:1009100078F001C077F000C076F037921CD071B249
:1009200002D0898201D08992898671724C506224EA
:10093000006E4D506320016E000E6420026E000EAA
:100940006520036E03C079F002C078F001C077F033
:1009500000C076F037827FD1020E6C5C3DE18B9057
:1009600039B405D07D687C687B687A6834D037A458
:1009700016D03E506224006E3F506320016E000E80
:100980006420026E000E6520036E03C07DF002C07D
:100990007CF001C07BF000C07AF037941CD071B4B9
:1009A00002D0898801D089988B8071744E5062245E
:1009B000006E4F506320016E000E6420026E000E28
:1009C0006520036E03C07DF002C07CF001C07BF0A7
:1009D00000C07AF037843FD1030E6C5C3DE18B920E
:1009E00039B605D0816980697F687E6834D037A6C2
:1009F00016D040506224006E41506320016E000EFC
:100A00006420026E000E6520036E03C081F002C0F8
:100A100080F001C07FF000C07EF037961CD071B628
:100A200002D0898A01D0899A8B82717650506224D3
:100A3000006E51506320016E000E6420026E000EA5
:100A40006520036E03C081F002C080F001C07FF01A
:100A500000C07EF03786FFD0040E6C5C3DE18B98C1
:100A600039B805D0856984698369826934D037A82B
:100A700016D042506224006E43506320016E000E77
:100A80006420026E000E6520036E03C085F002C074
:100A900084F001C083F000C082F037981CD071B898
:100AA00002D08B8401D08B948B8871785250622451
:100AB000006E53506320016E000E6420026E000E23
:100AC0006520036E03C085F002C084F001C083F08E
:100AD00000C082F03788BFD0050E6C5C3DE18B9A78
:100AE00039BA05D0896988698769866934D037AA97
:100AF00016D044506224006E45506320016E000EF3
:100B00006420026E000E6520036E03C089F002C0EF
:100B100088F001C087F000C086F0379A1CD071BA07
:100B200002D08B8601D08B968B8A717A54506224C6
:100B3000006E55506320016E000E6420026E000EA0
:100B40006520036E03C089F002C088F001C087F001
:100B500000C086F0378A7FD0060E6C5C3DE18A9437
:100B600039BC05D08D698C698B698A6934D037AC02
:100B700016D046506224006E47506320016E000E6E
:100B80006420026E000E6520036E03C08DF002C06B
:100B90008CF001C08BF000C08AF0379C1CD071BC77
:100BA00002D08A8001D08A908A84717C5650622457
:100BB000006E57506320016E000E6420026E000E1E
:100BC0006520036E03C08DF002C08CF001C08BF075
:100BD00000C08AF0378C3FD0070E6C5C3CE18A96EF
:100BE00039BE05D0916990698F698E6934D037AE6E
:100BF00016D048506224006E49506320016E000EEA
:100C00006420026E000E6520036E03C091F002C0E6
:100C100090F001C08FF000C08EF0379E1CD071BEE6
:100C200002D08A8201D08A928A86717E58506224CC
:100C3000006E59506320016E000E6420026E000E9B
:100C40006520036E03C091F002C090F001C08FF0E8
:100C500000C08EF0378E17D865AE0CD0656A646A16
:100C6000636A626A376A396A00EE72F0200EEE68D3
:100C7000E82EFDD706D065AE04D0656A646A636A63
:100C8000626A12EF01F06C686B8E0B6A080E0B5CE7
:100C900033E2D8900B34E96EEA6AEA36E936EA368E
:100CA000720EE926000EEA22EFCF00F0ECCF01F041
:100CB000ECCF02F0ECCF03F06850005C69500158B3
:100CC0006A5002586B50035815E2D8900B34E96E05
:100CD000EA6AEA36E936EA36720EE926000EEA22B8
:100CE000EFCF68F0ECCF69F0ECCF6AF0ECCF6BF0AF
:100CF0000BC06CF00B2ACAE312003A0E115C14E12F
:100D000012C05AF05A520CE003EE92F0D8905A34C6
:100D1000E926000EEA22EECF3AF0EFCF3BF003D007
:100D20003B6A3A6A3990A0D03B0E115C14E112C0C4
:100D30005BF05B520CE003EE92F0D8905B34E92656
:100D4000000EEA22EECF3CF0EFCF3DF003D03D6A3B
:100D50003C6A399289D03C0E115C14E112C05CF0FF
:100D60005C520CE003EE92F0D8905C34E926000E61
:100D7000EA22EECF3EF0EFCF3FF003D03F6A3E6A6B
:100D8000399472D03D0E115C14E112C05DF05D52D9
:100D90000CE003EE92F0D8905D34E926000EEA22D2
:100DA000EECF40F0EFCF41F003D0416A406A399670
:100DB0005BD03E0E115C14E112C05EF05E520CE09E
:100DC00003EE92F0D8905E34E926000EEA22EECFD0
:100DD00042F0EFCF43F003D0436A426A399844D0DF
:100DE0003F0E115C14E112C05FF05F520CE003EEA5
:100DF00092F0D8905F34E926000EEA22EECF44F05C
:100E0000EFCF45F003D0456A446A399A2DD0400EA1
:100E1000115C14E112C060F060520CE003EE92F03D
:100E2000D8906034E926000EEA22EECF46F0EFCFEC
:100E300047F003D0476A466A399C16D0410E115CD0
:100E400013E112C061F061520CE003EE92F0D89011
:100E50006134E926000EEA22EECF48F0EFCF49F0E8
:100E600003D0496A486A399E116812001668120058
:100E70001E0E135CD8A487D014521BE18A98396ADD
:100E80003B6A3A6A5A6A3D6A3C6A5B6A3F6A3E6AF2
:100E90005C6A416A406A5D6A436A426A5E6A456AA0
:100EA000446A5F6A476A466A606A496A486A616A70
:100EB00069D014C05AF003EE92F0D8901434E926A9
:100EC000000EEA22EECF3AF0EFCF3BF014C05BF019
:100ED00003EE92F0D8901434E926000EEA22EECF09
:100EE0003CF0EFCF3DF014C05CF003EE92F0D890F0
:100EF0001434E926000EEA22EECF3EF0EFCF3FF0A9
:100F000014C05DF003EE92F0D8901434E926000E80
:100F1000EA22EECF40F0EFCF41F014C05EF003EED6
:100F200092F0D8901434E926000EEA22EECF42F077
:100F3000EFCF43F014C05FF003EE92F0D89014347A
:100F4000E926000EEA22EECF44F0EFCF45F014C0C0
:100F500060F003EE92F0D8901434E926000EEA22F5
:100F6000EECF46F0EFCF47F014C061F003EE92F001
:100F7000D8901434E926000EEA22EECF48F0EFCFE5
:100F800049F08A881CD0420E135C07E1145203E139
:100F9000389017D801D0388012D07B0E135C0BE14B
:100FA000376A396A899489968B908B928B988B9A41
:100FB0008A948A9604D07F0E135CD8B426D813681E
:100FC0001200376A396A899489968B908B928B9834
:100FD0008B9A8A948A963B6A3A6A5A6A3D6A3C6A54
:100FE0005B6A3F6A3E6A5C6A416A406A5D6A436A5C
:100FF000426A5E6A456A446A5F6A476A466A606A2C
:10100000496A486A616A8A981200716A3B6A3A6A58
:101010005A6A3D6A3C6A5B6A3F6A3E6A5C6A416A38
:10102000406A5D6A436A426A5E6A456A446A5F6A08
:10103000476A466A606A496A486A616A4B6A4A6AEC
:101040004D6A4C6A4F6A4E6A516A506A536A526AD4
:10105000556A546A576A566A596A586A7568746854
:101060007368726879687868776876687D687C6884
:101070007B687A68816980697F687E688569846930
:101080008369826989698869876986698D698C69DC
:101090008B698A69916990698F698E697F0E6B6E21
:1010A0006A68696868686C68899089840A0E0DECC2
:1010B00000F08994899289860A0E0DEC00F08996D9
:1010C00089988B800A0E0DEC00F08B90899A8B82A8
:1010D0000A0E0DEC00F08B928B948B880A0E0DECAF
:1010E00000F08B988B968B8A0A0E0DEC00F08B9A91
:1010F0008A908A840A0E0DEC00F08A948A928A867D
:101100000A0E0DEC00F08A968A981200030193698A
:101110009269A20E956FC30E946F9A0E976F460E4A
:10112000966F960E996F320E986F920E9B6F3A0ED5
:101130009A6F8E0E9D6F5D0E9C6F8A0E9F6F9A0E3A
:101140009E6F860EA16FF00EA06F830EA36F5F0ED1
:10115000A26F7F0EA56FE70EA46F7C0EA76F850EA2
:10116000A66F790EA96F3B0EA86F760EAB6F070EB8
:10117000AA6F720EAD6FE80EAC6F6F0EAF6FDF0E21
:10118000AE6F6C0EB16FEA0EB06F6A0EB36F0A0EDF
:10119000B26F670EB56F3C0EB46F640EB76F820E00
:1011A000B66F610EB96FDA0EB86F5F0EBB6F440E8B
:1011B000BA6F5C0EBD6FBF0EBC6F5A0EBF6F4C0E88
:1011C000BE6F570EC16FE90EC06F550EC36F960EFE
:1011D000C26F530EC56FC46F510EC76F200EC66F1E
:1011E0004E0EC96FFB0EC86F4C0ECB6FE50ECA6F6B
:1011F0004A0ECD6FDC0ECC6F480ECF6FE20ECE6F75
:10120000460ED16FF50ED06F450ED36F150ED26F0F
:10121000430ED56F420ED46F410ED76F7B0ED66F43
:101220003F0ED96FC00ED86F3E0EDB6F100EDA6F17
:101230003C0EDD6F6D0EDC6F3A0EDF6FD40EDE6F8D
:10124000390EE16F460EE06F370EE36FC20EE26FAC
:10125000360EE56F490EE46F340EE76FDA0EE66F77
:10126000330EE96F740EE86F320EEB6F180EEA6FF3
:10127000300EED6FC50EEC6F2F0EEF6F7B0EEE6F25
:101280002E0EF16F3A0EF06F2D0EF36F020EF26F0D
:101290002B0EF56FD10EF46F2A0EF76FA90EF66FB5
:1012A000290EF96F880EF86F280EFB6F6F0EFA6F1C
:1012B000270EFD6F5E0EFC6F260EFF6F530EFE6F46
:1012C000250E0401016F500E006F240E036F540EA3
:1012D000026F230E056F5E0E046F220E076F6F0EF6
:1012E000066F210E096F860E086F200E0B6FA30E7E
:1012F0000A6F1F0E0D6FC60E0C6F1E0E0F6FEF0ED6
:101300000E6F1E0E116F106F1D0E136F520E126FA7
:101310001C0E156F8C0E146F1B0E176FCB0E166FF5
:101320001B0E196F0F0E186F1A0E1B6F580E1A6FC7
:10133000190E1D6FA50E1C6F180E1F6FF80E1E6F75
:10134000180E216F4F0E206F170E236FAB0E226FFA
:10135000170E256F0A0E246F160E276F6F0E266F5D
:10136000150E296FD70E286F150E2B6F430E2A6F9F
:10137000140E2D6FB30E2C6F140E2F6F270E2E6FC1
:10138000130E316F9F0E306F130E336F1A0E326FC4
:10139000120E356F990E346F120E376F1B0E366FAB
:1013A000110E396FA10E386F110E3B6F290E3A6F77
:1013B000100E3D6FB50E3C6F100E3F6F440E3E6F2A
:1013C0000F0E416FD60E406F0F0E436F6B0E426FC4
:1013D0000F0E456F030E446F0E0E476F9D0E466F46
:1013E0000E0E496F3A0E486F0D0E4B6FDA0E4A6FB4
:1013F0000D0E4D6F7C0E4C6F0D0E4F6F210E4E6F0C
:101400000C0E516FC80E506F0C0E536F720E526F50
:101410000C0E556F1E0E546F0B0E576FCC0E566F81
:101420000B0E596F7C0E586F0B0E5B6F2E0E5A6FA2
:101430000A0E5D6FE30E5C6F0A0E5F6F990E5E6FB2
:101440000A0E616F510E606F0A0E636F0B0E626FB2
:10145000090E656FC80E646F090E676F850E666FA3
:10146000090E696F450E686F090E6B6F060E6A6F85
:10147000080E6D6FC90E6C6F080E6F6F8E0E6E6F5B
:10148000080E716F540E706F080E736F1C0E726F22
:10149000070E756FE50E746F070E776FAF0E766FE0
:1014A000070E796F7B0E786F070E7B6F490E7A6F90
:1014B000070E7D6F170E7C6F060E7F6FE70E7E6F37
:1014C000060E816FB90E806F060E836F8B0E826FD2
:1014D000060E856F5F0E846F060E876F340E866F63
:1014E000060E896F0A0E886F050E8B6FE10E8A6FEC
:1014F000050E8D6FB90E8C6F050E8F6F930E8E6F6C
:10150000050E916F6D0E906F000112000201956B38
:101510002F0E946F976B340E966F996B390E986FF0
:101520009B6B3E0E9A6F9D6B420E9C6F9F6B470E9E
:101530009E6FA16B4C0EA06FA36B510EA26FA56B9B
:10154000560EA46FA76B5B0EA66FA96B600EA86FFB
:10155000AB6B650EAA6FAD6B690EAC6FAF6B6E0EA9
:10156000AE6FB16B730EB06FB36B780EB26FB56BBD
:101570007D0EB46FB76B820EB66FB96B870EB86F06
:10158000BB6B8C0EBA6FBD6B900EBC6FBF6B950EB4
:10159000BE6FC16B9A0EC06FC36B9F0EC26FC56BDF
:1015A000A40EC46FC76BA90EC66FC96BAE0EC86F11
:1015B000CB6BB30ECA6FCD6BB70ECC6FCF6BBC0EBF
:1015C000CE6FD16BC10ED06FD36BC60ED26FD56B01
:1015D000CB0ED46FD76BD00ED66FD96BD50ED86F1C
:1015E000DB6BDA0EDA6FDD6BDE0EDC6FDF6BE30ECA
:1015F000DE6FE16BE80EE06FE36BED0EE26FE56B23
:10160000F20EE46FE76BF70EE66FE96BFC0EE86F26
:10161000010EEB6FEA6FED6F050EEC6F010EEF6FD1
:101620000A0EEE6F010EF16F0F0EF06F010EF36FE9
:10163000140EF26F010EF56F190EF46F010EF76FB5
:101640001E0EF66F010EF96F230EF86F010EFB6F81
:10165000280EFA6F010EFD6F2C0EFC6F010EFF6F4E
:10166000310EFE6F010E0301016F360E006F010E89
:10167000036F3B0E026F010E056F400E046F010EEB
:10168000076F450E066F010E096F4A0E086F010EB7
:101690000B6F4F0E0A6F010E0D6F530E0C6F010E84
:1016A0000F6F580E0E6F010E116F5D0E106F010E51
:1016B000136F620E126F010E156F670E146F010E1D
:1016C000176F6C0E166F010E196F710E186F010EE9
:1016D0001B6F760E1A6F010E1D6F7A0E1C6F010EB6
:1016E0001F6F7F0E1E6F010E216F840E206F010E83
:1016F000236F890E226F010E256F8E0E246F010E4F
:10170000276F930E266F010E296F980E286F010E1A
:101710002B6F9D0E2A6F010E2D6FA10E2C6F010EE7
:101720002F6FA60E2E6F010E316FAB0E306F010EB4
:10173000336FB00E326F010E356FB50E346F010E80
:10174000376FBA0E366F010E396FBF0E386F010E4C
:101750003B6FC40E3A6F010E3D6FC80E3C6F010E19
:101760003F6FCD0E3E6F010E416FD20E406F010EE6
:10177000436FD70E426F010E456FDC0E446F010EB2
:10178000476FE10E466F010E496FE60E486F010E7E
:101790004B6FEB0E4A6F010E4D6FEF0E4C6F010E4B
:1017A0004F6FF40E4E6F010E516FF90E506F010E18
:1017B000536FFE0E526F020E556F030E546F020EE2
:1017C000576F080E566F020E596F0D0E586F020EAE
:1017D0005B6F120E5A6F020E5D6F160E5C6F020E7B
:1017E0005F6F1B0E5E6F020E616F200E606F020E48
:1017F000636F250E626F020E656F2A0E646F020E14
:10180000676F2F0E666F020E696F340E686F020EDF
:101810006B6F390E6A6F020E6D6F3D0E6C6F020EAC
:101820006F6F420E6E6F020E716F470E706F020E79
:10183000736F4C0E726F020E756F510E746F020E45
:10184000776F560E766F020E796F5B0E786F020E11
:101850007B6F600E7A6F020E7D6F640E7C6F020EDE
:101860007F6F690E7E6F020E816F6E0E806F020EAB
:10187000836F730E826F020E856F780E846F020E77
:10188000876F7D0E866F020E896F820E886F020E43
:101890008B6F870E8A6F020E8D6F8B0E8C6F020E10
:1018A0008F6F900E8E6F020E916F950E906F010EDE
:1018B0000B6E0001800E0B5C1DE202EE92F0D890E0
:1018C0000B34E926000EEA22EECF04F0EFCF05F04C
:1018D000D8900434006E0534016E02EE92F0D89078
:1018E0000B34E926000EEA2200C0EEFF01C0EFFF34
:0818F0000B2ADFE31200FFD711
:020000040030CA
:0300010006160ED2
:020005008580F4
:060008000FC00FE00F40E5
:00000001FF
